:100000000C945E060C94951D0C946E1D0C94860643
:100010000C9486060C9408200C9486060C94DA1F27
:100020000C94331F0C9486060C9486060C9486065A
:100030000C9486060C9486060C9486060C94860610
:100040000C94241D0C9486060C94E21D0C94BC1D8B
:100050000C9486060C9486060C9486060C948606F0
:100060000C94141E0C94860668031801726818809C
:10007000234020034C69676874734F4E04034F4E4E
:10008000042020202020BE5004B03B805F50046834
:100090003B0205680576380A01285004683B282F82
:1000A0006805183802004F680576380A00295004A0
:1000B000683B212650046832101E50046832111F1C
:1000C000C004BF1103696804800200EE8003680168
:1000D000EA1804FF0200E16804C00200AEC0036831
:1000E00001AA681880234020032041555820492F39
:1000F0005004032020042020202020E968188023B9
:10010000402003425420417564696F040320200499
:100110002020202020F368188023402003555342DC
:10012000617564696F04032020042020202020A131
:1001300068188023402003432E2044697363200401
:10014000032020042020202020C368188023402082
:1001500003464D20626E64203104032020042020D9
:10016000202020C1681880234020034C6F6E6777E1
:1001700061766504032020042020202020BC68181C
:1001800080234020034D2E205761766520040320F4
:1001900020042020202020D56818802340200346FA
:1001A0004D20426E642033040320200420202020B0
:1001B00020E368188023402003464D20626E6420AF
:1001C0003204032020042020202020C26805183893
:1001D00003004E68057638030020180A68390209C2
:1001E000003F000101776805183801004C0000004D
:1001F00000003E5B4F5B3E3E6B4F6B3E1C3E7C3EC9
:100200001C183C7E3C181C577D571C1C5E7F5E1CD6
:1002100000183C1800FFE7C3E7FF0018241800FF90
:10022000E7DBE7FF30483A060E2629792926407F8A
:10023000050507407F05253F5A3CE73C5A7F3E1C99
:100240001C08081C1C3E7F14227F22145F5F005F85
:100250005F06097F017F006689956A606060606063
:1002600094A2FFA29408047E040810207E201008A7
:10027000082A1C08081C2A08081E101010100C1E42
:100280000C1E0C30383E3830060E3E0E06000000C4
:10029000000000005F00000007000700147F147FCB
:1002A00014242A7F2A1223130864623649562050E8
:1002B0000008070300001C2241000041221C002A04
:1002C0001C7F1C2A08083E080800807030000808BF
:1002D000080808000060600020100804023E514930
:1002E000453E00427F400072494949462141494DFF
:1002F000331814127F1027454545393C4A49493186
:1003000041211109073649494936464949291E0004
:1003100000140000004034000000081422411414AE
:10032000141414004122140802015909063E415DCB
:10033000594E7C1211127C7F494949363E41414158
:10034000227F4141413E7F494949417F09090901D5
:100350003E414151737F0808087F00417F410020E2
:1003600040413F017F081422417F404040407F02CE
:100370001C027F7F0408107F3E4141413E7F0909F6
:1003800009063E4151215E7F0919294626494949FE
:100390003203017F01033F4040403F1F2040201FA8
:1003A0003F4038403F63140814630304780403613A
:1003B00059494D43007F414141020408102000414A
:1003C00041417F04020102044040404040000307D5
:1003D000080020545478407F28444438384444442A
:1003E00028384444287F385454541800087E0902A1
:1003F00018A4A49C787F0804047800447D40002061
:1004000040403D007F1028440000417F40007C04B4
:100410007804787C080404783844444438FC182470
:10042000241818242418FC7C080404084854545444
:100430002404043F44243C4040207C1C2040201CD9
:100440003C4030403C44281028444C9090907C44E0
:1004500064544C440008364100000077000000411D
:1004600036080002010204023C2623263C1EA1A1FC
:1004700061123A4040207A385454555921555579E3
:1004800041225454784221555478402054557940A3
:100490000C1E527212395555555939545454593904
:1004A000555454580000457C410002457D420001EE
:1004B000457C407D1211127DF0282528F07C545592
:1004C00045002054547C547C0A097F4932494949EB
:1004D000323A4444443A324A4848303A4141217A17
:1004E0003A42402078009DA0A07D3D4242423D3DE1
:1004F0004040403D3C24FF2424487E4943662B2F46
:10050000FC2F2BFF0929F620C0887E0903205454B4
:1005100079410000447D413048484A323840402209
:100520007A007A0A0A727D0D19317D2629292F2831
:10053000262929292630484D40203808080808086F
:10054000080808382F10C8ACBA2F102834FA000059
:100550007B000008142A142222142A14085500557E
:100560000055AA55AA55AAFF55FF55FF000000FFE8
:1005700000101010FF00141414FF001010FF00FFF3
:100580001010F010F0141414FC001414F700FF0005
:1005900000FF00FF1414F404FC141417101F1010B3
:1005A0001F101F1414141F00101010F00000000082
:1005B0001F101010101F10101010F010000000FF7E
:1005C000101010101010101010FF10000000FF1479
:1005D0000000FF00FF00001F10170000FC04F414CF
:1005E000141710171414F404F40000FF00F7141487
:1005F0001414141414F700F7141414171410101F03
:10060000101F141414F4141010F010F000001F1038
:100610001F0000001F14000000FC140000F010F088
:100620001010FF10FF141414FF141010101F0000FE
:100630000000F010FFFFFFFFFFF0F0F0F0F0FFFF11
:10064000FF0000000000FFFF0F0F0F0F0F384444A2
:100650003844FC4A4A4A347E02020606027E027E82
:100660000263554941633844443C04407E201E20C7
:1006700006027E020299A5E7A5991C2A492A1C4C6C
:100680007201724C304A4D4D303048784830BC626F
:100690005A463D3E494949007E0101017E2A2A2AE7
:1006A0002A2A44445F444440514A444040444A5109
:1006B000400000FF0103E080FF000008086B6B08AA
:1006C0003612362436060F090F06000018180000EF
:1006D000001010003040FF0101001F01011E001931
:1006E0001D1712003C3C3C3C0000000000000103D0
:1006F000070F1F3F7F0080C0E0F0F8FCFEDB40A446
:10070000A62EAF2000A1C8D300408DAED580A80092
:100710000060000000000000000000000000000079
:10072000E00000000000000000000000000001E008
:100730000000000000000000000000000001F000C8
:1007400000000000000000000000000003F00000B6
:10075000000000000000000000000007F0000000A2
:100760000000000000000000000007F8000000008A
:100770000000000000000000000FF800000003C0AF
:10078000007E000001E0007F0FF800000003C000C1
:10079000FE000001E000FFEFF800000003C000FED3
:1007A000000001E000FFFFF800000003C000F000BF
:1007B00000000F007FFE7FC0000003C000F00000BB
:1007C000000F003FFE7FF83FF1FBCFFCFEF3BC3D86
:1007D000EFE01FFE7FFF7FFBFFDFFEFEFFBC3DEF74
:1007E000E01FC6FFFF7FFBFFDFFEFEFFBC3DEFE02B
:1007F0000FE3C7FE787BC3DE1EF0FFBC3DEF0007B2
:10080000FF87FC787BC3DE1EF0F83C3DEF0001FF64
:10081000FFF0007BC3C01EF0F03C3DEF0001F37F12
:10082000E03FFBC3CFFEF0F03C3DEF0003E33F8031
:100830007FFBC3DFFEF0F03C3DEF0007E73C0078B4
:100840007BC3DE1EF0F03C3DEF0007FFBE00787B6F
:10085000C3DE1EF0F03C3DEF0007FFFE00787BC3D7
:10086000DE1EF0F03C3DEF000FFFFE007FFBFFDFE0
:10087000FEF0F03FFDEFE00FFFFF007FFBFFDFFE2C
:10088000F0F03FFDEFE00FF9FF003E79F9CF9EF069
:10089000F01F3DE7E01FF1FF000000000000000036
:1008A000000000001F80FF007FFFFFFFFFFFFFFF32
:1008B000FFFFE01C007F007FFFFFFFFEB46D888D0F
:1008C00018E000001F007FFFFFFFFE95AD7DB577AC
:1008D000E000000F007FFFFFFFFEA5AD9D8D19E03A
:1008E000000006007FFFFFFFFEB5ADEDB57EE00026
:1008F0000000000001800000000000000000000374
:100900008000000000000000000007C000000000A0
:10091000000000000007C000000000000000000010
:100920000FC00000000000000000001FE0000000F9
:100930000000000000001FE00000000000000000B8
:10094000003FE00000000000000000003FF0000059
:10095000000000000000007FF00000000000000028
:100960001FF87FF0000000000000003FFE7FF00055
:100970000000000000003FFF7FF0000000000000CA
:10098000001FFFFBE0000000000000000FFFF9FF68
:10099000C00000000000000FFFF9FFF80000000099
:1009A000000007FFF1FFFF00000000000003FC73E0
:1009B000FFFF80000000000001FE3FFFFF800000FD
:1009C00000000000FF1E0FFF000000000000007F7D
:1009D000FE1FFC000000000000003FFFFFF80000C9
:1009E00000000000000FDFFFE0000000000000003A
:1009F0001F19FFC0000000000000003F3CFF000086
:100A00000000000000007E7CF800000000000000F4
:100A1000007FFE7C0000000000000000FFFFFC00E3
:100A200000000000000000FFFFFE000000000000CA
:100A30000000FFFFFE0000000000000001FFEFFECD
:100A40000000000000000001FFCFFE0000000000D9
:100A5000000003FF07FE0000000000000003FC0789
:100A6000FE0000000000000003F003FE0000000094
:100A7000000000018000FE000000000000000000F7
:100A8000007E000000000000000000003E000000AA
:100A9000000000000000000C0000000000000780C3
:100AA00000FC000003C0000000078001FC00000300
:100AB000C0000000078001FC000003C00000000728
:100AC0008001E00000001E000000078001E000003F
:100AD000001E007FE3F79FF9FDE7787BDFC0FFF79B
:100AE000FFBFFDFDFF787BDFC0FFF7FFBFFDFDFF10
:100AF000787BDFC0F0F787BC3DE1FF787BDE00F05C
:100B0000F787BC3DE1F0787BDE0000F787803DE1B0
:100B1000E0787BDE007FF7879FFDE1E0787BDE00F9
:100B2000FFF787BFFDE1E0787BDE00F0F787BC3D93
:100B3000E1E0787BDE00F0F787BC3DE1E0787BDE2A
:100B400000F0F787BC3DE1E0787BDE00FFF7FFBFF8
:100B5000FDE1E07FFBDFC0FFF7FFBFFDE1E07FFBD2
:100B6000DFC07CF3F39F3DE1E03E7BCFC00000009F
:100B70000000000000000000FFFFFFFFFFFFFFFF7D
:100B8000FFFFC0FFFFFFFFFD68DB111A31C0FFFF51
:100B9000FFFFFD2B5AFB6AEFC0FFFFFFFFFD4B5B22
:100BA0003B1A33C0FFFFFFFFFD6B5BDB6AFDC057E5
:100BB000616974696E6720666F7220492D42757392
:100BC0000053706565642F52504D206D6F6E6974CF
:100BD0006F72004149204D6F64756C65203132455C
:100BE000005353443133303620616C6C6F63617451
:100BF000696F6E206661696C65640052504D3A20E1
:100C000000206B6D2F68004D65747269633A200097
:100C1000202041637475616C3A2000202053796E66
:100C20006320553A2000202053796E6320443A20F7
:100C30000020204175746F3A204F4646005461727F
:100C40006765743A2000204D504800537065656414
:100C50003A20006804BF0201D000000000240027F1
:100C6000002A0000000000250028002B00000000E2
:100C7000080002010000030407000000000000005B
:100C8000002200FF210000000023002600290004AC
:100C90000404040404040402020202020203030323
:100CA000030303010204081020408001020408101D
:100CB00020010204081020008A20552011241FBEA4
:100CC000CFEFD8E0DEBFCDBF25E0A4EAB1E001C0A0
:100CD0001D92A433B207E1F711E0A0E0B1E0E8EA29
:100CE000F5E502C005900D92A43AB107D9F716E0D8
:100CF000CDE5D6E004C02197FE010E948729CC35BE
:100D0000D107C9F70E94B3210C94C72A0C940000A4
:100D10000895833081F028F4813099F08230A9F071
:100D200008958730A9F08830C9F08430B1F48091FB
:100D300080008F7D03C0809180008F77809380003A
:100D4000089584B58F7784BD089584B58F7DFBCFDA
:100D50008091B0008F778093B00008958091B000AB
:100D60008F7DF9CFCF93DF93282F30E0F901E3593E
:100D7000F34F8491F901ED55F34FD491F901E15707
:100D8000F34FC491CC23A1F081110E948906EC2F6E
:100D9000F0E0EE0FFF1FEB57F34FA591B491EC91EC
:100DA000ED2381E090E009F480E0DF91CF91089598
:100DB00080E090E0FACF1F93CF93DF93282F30E0AD
:100DC000F901E359F34F8491F901ED55F34FD491B3
:100DD000F901E157F34FC491CC23A9F0162F8111EB
:100DE0000E948906EC2FF0E0EE0FFF1FED59F34F44
:100DF000A591B4918FB7F894EC91111108C0D095DA
:100E0000DE23DC938FBFDF91CF911F910895DE2BFE
:100E1000F8CFCF93DF9390E0FC01ED55F34F249191
:100E20008157934FFC0184918823C9F090E0880F8B
:100E3000991FFC01E75AF34FA591B491FC01ED59BC
:100E4000F34FC591D49161110DC09FB7F8948C9167
:100E5000209582238C938881282328839FBFDF914C
:100E6000CF910895623051F49FB7F8943C91822F4E
:100E7000809583238C93E8812E2BEFCF8FB7F89446
:100E8000EC912E2B2C938FBFEACF3FB7F894809133
:100E90007F0290918002A0918102B091820226B5DA
:100EA000A89B05C02F3F19F00196A11DB11D3FBFA2
:100EB000BA2FA92F982F8827BC01CD01620F711D71
:100EC000811D911D42E0660F771F881F991F4A956B
:100ED000D1F708958F929F92AF92BF92CF92DF92F7
:100EE000EF92FF924B015C010E9445076B017C0170
:100EF0000E9445076C197D098E099F09683E734061
:100F000081059105A8F321E0821A9108A108B10892
:100F100088EEC80E83E0D81EE11CF11C81149104F8
:100F2000A104B10429F7FF90EF90DF90CF90BF901C
:100F3000AF909F908F9008952FB7F89460917B02A7
:100F400070917C0280917D0290917E022FBF089566
:100F50000895089508950895EF92FF920F931F93B7
:100F6000CF93DF938C017B01D0E0C0E0F701EC0F61
:100F7000FD1F6491662361F0D801ED91FC91019011
:100F8000F081E02DC8010995892B11F02196EECF53
:100F9000CE01DF91CF911F910F91FF90EF900895B7
:100FA000AF92BF92CF92DF92EF92FF920F931F9377
:100FB000CF93DF936C017B018B01040F151FEB01B5
:100FC0005E01AE18BF08C017D10759F06991D6016C
:100FD000ED91FC910190F081E02DC6010995892BDE
:100FE00079F7C501DF91CF911F910F91FF90EF909D
:100FF000DF90CF90BF90AF900895FC01538D448D4A
:10100000252F30E0842F90E0821B930B541710F0B3
:10101000CF96089501970895FC01918D828D9817C0
:1010200061F0A28DAE0FBF2FB11D5D968C91928D98
:101030009F5F9F73928F90E008958FEF9FEF0895C9
:10104000FC01918D828D981731F0828DE80FF11D92
:10105000858D90E008958FEF9FEF0895FC01918DAD
:10106000228D892F90E0805C9F4F821B91098F73A6
:101070009927089587E892E00E942E0821E0892BA5
:1010800009F420E0822F089580E090E0892B29F078
:101090000E943A0881110C9400000895FC01A48D6F
:1010A000A80FB92FB11DA35ABF4F2C91848D90E08A
:1010B00001968F739927848FA689B7892C93A0896D
:1010C000B1898C91837080648C93938D848D9813F7
:1010D00006C00288F389E02D80818F7D808308958A
:1010E000EF92FF920F931F93CF93DF93EC0181E078
:1010F000888F9B8D8C8D98131AC0E889F98980811F
:1011000085FF15C09FB7F894EE89FF896083E88951
:10111000F98980818370806480839FBF81E090E043
:10112000DF91CF911F910F91FF90EF900895F62ED0
:101130000B8D10E00F5F1F4F0F731127E02E8C8D6A
:101140008E110CC00FB607FCFACFE889F9898081AF
:1011500085FFF5CFCE010E944E08F1CFEB8DEC0F4D
:10116000FD2FF11DE35AFF4FF0829FB7F8940B8FCC
:10117000EA89FB8980818062CFCFCF93DF93EC0136
:10118000888D8823B9F0AA89BB89E889F9898C916F
:1011900085FD03C0808186FD0DC00FB607FCF7CF2B
:1011A0008C9185FFF2CF808185FFEDCFCE010E942B
:1011B0004E08E9CFDF91CF910895EF92FF920F9300
:1011C0001F93CF93DF93EC01EC80FD806E157F05BC
:1011D0000CF070C057FF04C0240F351F50E040E0F2
:1011E0008E819F81FA01E20FF31F8E179F071CF477
:1011F0009C01241B350B121613060CF05BC0922FBA
:10120000842F8695869586958E9DD0018F9DB00DF5
:1012100011246A0F7B1FAF8DB8A1A60FB71F4770AF
:1012200049F188E0841B482F682F70E0FB01EB50E8
:10123000F94FE491281708F063C0621B71092FEF82
:1012400030E002C0359527956A95E2F7E223013038
:10125000110539F0B0F10230110561F58C91E827E4
:1012600002C08C91E82BEC93941720F12C813D81E6
:10127000A20FB31FE92FE41BE83078F0023011050C
:1012800021F58E2F9C9190959C932C813D81A20FEE
:10129000B31F88508830B0F7E770EE2359F0F0E0C4
:1012A000E351F94FE49101301105F9F010F10230EA
:1012B000110519F1DF91CF911F910F91FF90EF90E0
:1012C0000895E0958C91E823CECF81E001151105BA
:1012D00009F480E081959E2F8C932C813D81A20F93
:1012E000B31F98509830C0F7D7CF8C91E82BEC9370
:1012F000E1CFE0958C91E823FACF8C91E827F7CFE6
:101300000130110509F4ADCFE0F20230110509F406
:10131000A5CFAE0DBF1DAECF0F931F93CF93DF931D
:1013200077FF04C0260F371F70E060E0DC011496E1
:10133000CD91DC91FB01E20FF31FCE17DF071CF408
:101340009E01261B370B121613064CF5FA0157FDAA
:101350003796A3E0F595E795AA95E1F7EC9FD001C4
:10136000ED9FB00DFC9FB00D11246A0F7B1FDC01B7
:101370005F96ED91FC91E60FF71F4770552781E0CE
:1013800090E001C0880F4A95EAF7482F0130110517
:1013900059F0A8F02E0F3F1F02301105E1F0DF9148
:1013A000CF911F910F9108952E0F3F1FE217F30762
:1013B000B1F38191DF011197842B8C93F7CF809546
:1013C0002E0F3F1FE217F30751F39191DF011197A1
:1013D00098239C93F7CFE217F30709F38191DF017C
:1013E000119784278C93F7CF0F931F93FA01DC0199
:1013F00056964C9156974230E9F04330A1F1413076
:1014000061F514964D915C91DA01AE1BBF0BFD01A5
:10141000E21BF30B77FD0BC0DC0116964D915C913E
:101420006417750724F4AB01BF010E948C091F915A
:101430000F91089514964D915C91DA01A61BB70B9C
:10144000BD0161507109DC0116964D915C91DA0184
:10145000AE1BBF0BFD01E21BF30B77FDE8CFAF0125
:101460000E94DD08E4CF16964D915C91DA01A61B2F
:10147000B70BBD0161507109CDCF0F931F93FA01D6
:10148000DC0156964C9156974230A9F0433091F1C9
:10149000413019F514964D915C91DA01AE1BBF0BEA
:1014A000FD013197F7FD04C0AB01BF010E94DD08CB
:1014B0001F910F91089514964D915C91DA01A61B2E
:1014C000B70BBD01DC0116964D915C91DA01AE1BA4
:1014D000BF0BFD013197621B730BF7FDE9CFDC01F8
:1014E00016964D915C91E417F50714F7AF010E9431
:1014F0008C09DECF16964D915C91DA01A61BB70BD5
:10150000BD01621B730BCECFFC0177FD64C08085EB
:101510009185681779070CF05EC057FD5CC0828525
:101520009385481759070CF056C086898230B1F070
:10153000833029F1813041F484819581841B950B9E
:10154000AB01BC01615071092130310509F108F48A
:1015500043C02230310509F463C008958481958128
:10156000DC01A61BB70BBD01615071098681978113
:10157000DC01A41BB50BAD0141505109E5CF8681BB
:101580009781861B970BBA01AC0141505109DCCF02
:10159000CA0157FD0796A3E095958795AA95E1F7AF
:1015A000A481B5818A9F90018B9F300D9A9F300D49
:1015B0001124620F731F078CF0A1E02DE60FF71FB7
:1015C0004770552721E030E001C0220F4A95EAF725
:1015D0008081822B80830895CA0157FD079633E0EE
:1015E000959587953A95E1F7A481B5818A9F9001F9
:1015F0008B9F300D9A9F300D1124620F731F078C43
:10160000F0A1E02DE60FF71F4770552781E090E02D
:1016100001C0880F4A95EAF7809590818923DACF37
:10162000CA0157FD079623E0959587952A95E1F71E
:10163000A481B5818A9F90018B9F300D9A9F300DB8
:101640001124620F731F078CF0A1E02DE60FF71F26
:101650004770552721E030E001C0220F4A95EAF794
:1016600080818227B7CF08958EBD00000DB407FE9C
:10167000FDCF8EB508958CBD9DBD08950895FC01E4
:101680006370668B8481958126813781613039F062
:10169000633029F0918780873387228708953187C7
:1016A00020879387828708952F923F924F925F926F
:1016B0006F927F928F929F92AF92BF92CF92DF9262
:1016C000EF92FF920F931F93CF93DF93CDB7DEB7C7
:1016D0006A970FB6F894DEBF0FBECDBF9A8F898F81
:1016E0007A8369834A01D22E18870F833701BC2C75
:1016F000DC0159962D913C915A972115310509F03D
:1017000015C118968D919C911997681779070CF05F
:10171000D7C11A968D919C91481759070CF0D0C1EA
:101720004C2C512CB6E0CB9E600D711D11247C8792
:101730006B87161617060CF0C3C1EA2DF0E0FA8786
:10174000E98793E0EE0FFF1F9A95E1F7F88BEF879B
:10175000CF01840F951F181619060CF0B1C1A98D81
:10176000BA8D58968C91811104C0BFEABD1508F45A
:10177000D394A98DBA8DED91FC9111970284F385D4
:10178000E02DCD010995B5E0DB9EC0011124E98172
:10179000FA81FC83EB83312C212C9C0123513E4F99
:1017A000388F2F8B4A2D50E05E8B4D8BEF89F88D53
:1017B000E20DF31D44919E828D82D12CC12C698152
:1017C0007A81620D731D7A8B698B842F90E09C8BDC
:1017D0008B8BE98DFA8DA081B18140FF82C0F1E051
:1017E000BF126FC0AF126DC01C96ED91FC912F819E
:1017F0003885A4014C0D5D1D69897A89898D9A8D82
:101800000995EB89FC89F595E7954E2F5FEFC51A91
:10181000D50A6D817E818D899E89680F791F7E83AF
:101820006D8398E0C916D10481F6AFEF2A1A3A0AFF
:10183000EB81FC81E40DF51DFC83EB83F5E02F16B5
:10184000310409F0B3CF2F81388526153705B9F05B
:10185000A98DBA8DED91FC91B1E0BB1257C0AB12CE
:1018600055C069817A816B5F7F4F0088F189E02DD7
:10187000830128E030E0A401898D9A8D0995A98D16
:10188000BA8DED91FC9111970688F789E02DCD0175
:101890006A960FB6F894DEBF0FBECDBFDF91CF9131
:1018A0001F910F91FF90EF90DF90CF90BF90AF907E
:1018B0009F908F907F906F905F904F903F902F9070
:1018C00009941E96ED91FC91EF80F88409851A85A4
:1018D00092014D815E816B817C81898D9A8D099504
:1018E00090CF2F8138852615370509F48ACF31E04E
:1018F000B31207C0A31205C01C96ED91FC91930191
:1019000078CF1E96ED91FC917301E0CF6B857C85BD
:10191000641975090684F785E02D73010F85188910
:101920009201A401898D9A8D0995A9CFF901349668
:101930009491329745915491D91AB7E0DB9E400DAE
:10194000511D1124F901259134913C8B2B8BFA0107
:1019500025903490FA013296749031963491398BF7
:10196000329664903196449041E04C1518F04A1537
:1019700008F07FC0662D062C000C770B7C836B83F0
:10198000842D042C000C990B9E838D83A98DBA8D18
:10199000ED91FC9111970284F385E02DCD0109951D
:1019A000512CD12CC12CEA2DF0E0FA87E9872B2DA0
:1019B00030E03C872B87A401440D511D47FC5A950C
:1019C000588F4F8B69817A81660D711D67FC7A95FE
:1019D0007E876D877989C71608F051CF2C2D30E0AE
:1019E0004D815E81420F531FA985BA854A9FC00170
:1019F0004B9F900D5A9F900D1124FC01E80DF91D8D
:101A0000F88BEF87852D612C4F89588D420F531F1E
:101A10005E8B4D8B671408F050C044244394480EED
:101A2000877041F4C1010196EB89FC89E20DF31D39
:101A3000D4901C01D7FE19C0A98DBA8DED91FC91EF
:101A4000662D70E0B1E0BB1219C0AB1217C02D8536
:101A50003E85620F731F0484F585E02D2F81388544
:101A60004D895E89898D9A8D0995DD0C6394842D4D
:101A7000D1CF1E821D821C821B8288CF4B815C814C
:101A8000640F751FAB85BC856A9FC0016B9F900D6D
:101A90007A9F900D112469817A81680F791F0684DD
:101AA000F785E02DEF80F88409851A859D014F8523
:101AB0005889898D9A8D0995D8CF570CC3948ACFB0
:101AC0006A960FB6F894DEBF0FBECDBFDF91CF91FF
:101AD0001F910F91FF90EF90DF90CF90BF90AF904C
:101AE0009F908F907F906F905F904F903F902F903E
:101AF00008958F929F92AF92CF92EF92FF920F93A1
:101B00001F93CF93DF93EC01262F898D9A8D009739
:101B100009F051C06A30D1F41D861C868D8948E0D9
:101B2000849F900111248E859F85820F931F9F872C
:101B30008E8781E090E0DF91CF911F910F91FF9010
:101B4000EF90CF90AF909F908F9008956D3089F374
:101B5000CC88AD888F898823C1F08C859D8536E03F
:101B6000C39E800D911D112448855985481759073A
:101B700064F44E855F851D861C8638E0A39EC001F7
:101B80001124840F951F9F878E87EA88FB88088918
:101B900019894E855F856C857D85CE010E94540B29
:101BA0002C898C859D8546E0249F800D911D1124F4
:101BB0009D878C87BECF6A3069F41D861C86FC0128
:101BC0003896E4912D898E859F85E29F800D911D29
:101BD0001124ADCF6D3009F4ACCFFC0134963491B3
:101BE000631708F4A6CF3296E491E61708F4A1CF64
:101BF000FC01329685909490462F431B342F47E08A
:101C0000349F800C911C1124F4013296349131964A
:101C1000E4913323A9F1EE2399F1CC88F4013596B0
:101C2000E491AD884F89442301F10E2E000CFF0B87
:101C3000E30FF11DCE9EA001CF9E500D11246C85A7
:101C40007D85460F571F68857985641775076CF485
:101C50004E855F851D861C86FC013896E491AE9EFC
:101C6000400D511D11245F874E87EA88FB88088943
:101C700019894E855F856C857D85CE010E94540B48
:101C8000F4013496E4912C898C859D85E29F800D2A
:101C9000911D11248DCF6F927F928F929F92AF9260
:101CA000BF92CF92DF92EF92FF920F931F93CF9349
:101CB000DF93EC016B015A0139014801E881F98198
:101CC0000284F385E02D0995E881F9810288F38982
:101CD000E02D87019301A501B601CE010995A5016B
:101CE000480D591D41505109E881F9810288F38955
:101CF000E02D9301B601CE010995E881F9810088B4
:101D0000F189E02D9401A501B601CE010995C60C1B
:101D1000D71CB60161507109E881F9810088F18909
:101D2000E02D9401A501CE010995E881F98106888D
:101D3000F789E02DCE01DF91CF911F910F91FF9098
:101D4000EF90DF90CF90BF90AF909F908F907F905B
:101D50006F9009946F927F928F929F92AF92BF92F1
:101D6000CF92DF92EF92FF920F931F93CF93DF9367
:101D70005C01EB016A01490138018701DC01ED9149
:101D8000FC916217730719F5641675062CF0962DF1
:101D9000872D3A01C92ED82E9601261937092F5FB3
:101DA0003F4F048CF58DE02DA301BE01C5010995BF
:101DB000DF91CF911F910F91FF90EF90DF90CF9027
:101DC000BF90AF909F908F907F906F900895461531
:101DD000570591F42617370724F0892D4B01C22FA0
:101DE000D82F9E01281939092F5F3F4F068CF78D98
:101DF000E02DA601B401DACF0284F385E02D099528
:101E0000D501ED91FC910488F589E02D83019401C1
:101E1000A601BE01C5010995D501ED91FC91068889
:101E2000F789E02DC501DF91CF911F910F91FF90B0
:101E3000EF90DF90CF90BF90AF909F908F907F906A
:101E40006F900994EF92FF920F931F93DC011A9603
:101E50000D911C911B9718962D913C911997ED911E
:101E6000FC9100A0F1A1E02D7B0150E040E070E08A
:101E700060E009951F910F91FF90EF9008954F92A8
:101E80005F926F927F928F929F92AF92BF92CF920A
:101E9000DF92EF92FF920F931F93CF93DF936C012A
:101EA0002B015A0139014801DC01ED91FC910284BA
:101EB000F385E02D0995E201640C751CD601ED91C6
:101EC000FC91C615D7055CF40088F189E02D8701E7
:101ED0009401A501BE01C60109952196EFCF0688A0
:101EE000F789E02DC601DF91CF911F910F91FF90EF
:101EF000EF90DF90CF90BF90AF909F908F907F90AA
:101F00006F905F904F9009948F929F92AF92BF9283
:101F1000CF92DF92EF92FF920F931F93CF93DF93B5
:101F2000EC015B014A016901E881F9810284F385D2
:101F3000E02D099595012C0D3D1D21503109E881B9
:101F4000F9810488F589E02D78018401A401B501A7
:101F5000CE010995E881F9810688F789E02DCE0147
:101F6000DF91CF911F910F91FF90EF90DF90CF9075
:101F7000BF90AF909F908F9009948F929F92AF9255
:101F8000BF92CF92DF92EF92FF920F931F93CF9366
:101F9000DF93EC015B014A0169017801E881F98175
:101FA0000284F385E02D0995C80CD91C86010150E7
:101FB0001109E881F9810488F589E02D9501A401D2
:101FC000B501CE010995E881F9810688F789E02DF0
:101FD000CE01DF91CF911F910F91FF90EF90DF9095
:101FE000CF90BF90AF909F908F900994EF92FF9207
:101FF0000F931F93DC01ED91FC9100A0F1A1E02D66
:1020000009951F910F91FF90EF9008950F931F93E3
:10201000DC01ED91FC91068CF78DE02D09951F9167
:102020000F9108950F931F93DC01ED91FC91048CA7
:10203000F58DE02D09951F910F910895DC01ED912B
:10204000FC910084F185E02D09943F924F925F92BC
:102050006F927F928F929F92AF92BF92CF92DF92B8
:10206000EF92FF920F931F93CF93DF935C017B015D
:102070004A016901390187E0680E711C93E075948B
:1020800067949A95E1F72B01400E511E10E000E095
:10209000312CD0E0C0E0CE0187709927330C892B1A
:1020A00059F4FE0183E0F595E7958A95E1F7E00F95
:1020B000F11FE80DF91D349037FE0AC021E030E031
:1020C000A701B5016C0F7D1F80EF94E00E941E10E8
:1020D0002196CC16DD06F9F68FEFE81AF80A060D00
:1020E000171DE414F504A9F6DF91CF911F910F910C
:1020F000FF90EF90DF90CF90BF90AF909F908F9028
:102100007F906F905F904F903F9008952F923F92F5
:102110004F925F926F927F928F929F92AF92BF92F7
:10212000CF92DF92EF92FF920F931F93CF93DF93A3
:1021300000D000D000D0CDB7DEB73C016A013E83AD
:102140002D83FC82EB825801A41AB50AB7FE03C0A6
:10215000B194A194B1088D809E80861A970A97FE4B
:1021600003C09194819491088A149B045CF0902F91
:10217000812F0D811E819D838E839C2D8D2D6B0162
:10218000692F782F0C151D055CF09D818E817E8353
:102190006D83692F782F902F812F8601C92ED82E1D
:1021A0001601201A310A2B012D813E81421A530A51
:1021B00057FE03C0519441945108710137FE03C08A
:1021C0003FEFE31AF30AF594E7948D819E81861719
:1021D00097075CF5A1E0B0E0BA83A983C016D106E9
:1021E0004CF1D301ED91FC910484F585E02D2B8118
:1021F0003C81A8016D817E818A149B041CF04D8175
:102200005E81B801C3010995E418F508F7FE0AC01C
:102210002D813E8189819A81280F391F3E832D832C
:10222000E20CF31C0F5F1F4FD9CF2FEF3FEF3A8324
:102230002983D4CF26960FB6F894DEBF0FBECDBF4C
:10224000DF91CF911F910F91FF90EF90DF90CF9092
:10225000BF90AF909F908F907F906F905F904F90C6
:102260003F902F900895089520911502260F33274F
:10227000331F21323105ECF420913902FC0190E04A
:1022800080E0243069F082E00895A0911502219148
:10229000AC014B505E4FA40FB52FB11D2C9301968E
:1022A000861798F380911502680F6093150280E0FD
:1022B000089581E008951092390281E080933B02F5
:1022C00010923A0261E082E10E94DB0661E083E164
:1022D0000E94DB06E9EBF0E080818E7F80838081C5
:1022E0008D7F808388E48093B80085E48093BC0070
:1022F0000895CF93DF9391E09093F4018823B9F090
:10230000C091B800D091BA008091BC008A7B8093C4
:10231000BC0060E082E10E94DB0660E083E10E9495
:10232000DB060E945B11D093BA00C093B800DF9126
:10233000CF910895E091650280916402E81730F42E
:10234000F0E0E153FE4F808190E008958FEF9FEF22
:10235000089590916502809164022FEF3FEF9817E6
:1023600048F4E92FF0E0E153FE4F208130E09F5F19
:1023700090936502C901089580916402909165026D
:10238000891B990B0895CF92DF92EF92FF920F93E2
:102390001F93CF93DF937C01CB018A0120918602AA
:1023A000222389F0EB016B01C40ED51ECC15DD058F
:1023B00069F06991D701ED91FC910190F081E02DD8
:1023C000C7010995F3CF642F0E943411C801DF9132
:1023D000CF911F910F91FF90EF90DF90CF900895D4
:1023E000CF93DF931F92CDB7DEB76983209186022A
:1023F0002223F9F020918302203258F021E030E0CE
:10240000FC013383228390E080E00F90DF91CF9135
:10241000089580918402E82FF0E0E155FE4F998104
:1024200090838F5F809384028093830281E090E0A9
:10243000ECCF61E0CE0101960E943411F7CFCF922C
:10244000DF92EF92FF920F931F93CF93DF93D09180
:10245000830281E0D13208F09CC0C09185020E94C5
:1024600045076B017C018091390281116CC082E0CB
:102470008093390281E080933B028FEF8093380292
:1024800010925D02D0935C02AFEAB1E0ECE3F2E0BF
:1024900080E0D8138DC010925E0280915E02CC0F56
:1024A000C82BC0935E0280913A02813009F084C04B
:1024B00010923A020E9445076B017C0180915E02F6
:1024C0008093BB008091F0019091F101A091F20105
:1024D000B091F301892B8A2B8B2BA1F00E94450729
:1024E0000091F0011091F1012091F2013091F3017E
:1024F0006C197D098E099F090617170728073907E8
:1025000008F442C08091BC0083FDD8CF85EC809355
:10251000BC000E9445076B017C018091390282302A
:1025200009F44CC0809138028F3F09F469C0809152
:102530003802803209F466C080913802803309F491
:1025400063C084E026C08091F0019091F101A091D8
:10255000F201B091F301892B8A2B8B2B09F483CFE5
:102560000E9445070091F0011091F1012091F201C4
:102570003091F3016C197D098E099F090617170721
:102580002807390708F06FCF8091EF010E94791179
:1025900085E0109284021092830210928602DF91ED
:1025A000CF911F910F91FF90EF90DF90CF90089502
:1025B0009D9191938F5F6DCF85EEA9CF8091F001B2
:1025C0009091F101A091F201B091F301892B8A2B36
:1025D0008B2B09F4A2CF0E9445070091F0011091C6
:1025E000F1012091F2013091F3016C197D098E09FE
:1025F0009F09061717072807390708F08ECFC4CFA1
:1026000080E0C7CF82E0C5CF83E0C3CFEF92FF92D7
:102610000F931F93CF93DF937C01C62F80910D05FD
:1026200090910E05009709F459C02091110531E0F1
:1026300030938602209385021092840210928302C6
:10264000DC01ED91FC910190F081E02D60E00995B5
:102650008701EE24E394F12CD1E0C15080910D0567
:1026600090910E05CF3F91F1B0E2EB16F104D8F056
:102670000E941F1280910D0590910E052091110569
:10268000D0938602209385021092840210928302D6
:10269000DC01ED91FC910190F081E02D60E0099565
:1026A000EE24E394F12C80910D0590910E05F80134
:1026B0006491DC01ED91FC910190F081E02D099590
:1026C000BFEFEB1AFB0A0F5F1F4FC7CFDF91CF9110
:1026D0001F910F91FF90EF900C941F12E0911D0538
:1026E000F0911E0590818091230580958923808338
:1026F0008701C15008F438C0F801849120910B057E
:1027000030910C05232B29F00E94340B0F5F1F4FD3
:10271000F0CF28E030E040E8E0911905F0911A058B
:1027200090912105582F5423D9F05081952B9083F7
:10273000E0911B05F0911C05908150912205952B8D
:102740009083E0911B05F0911C055081909122052A
:10275000909595239083469521503109E9F6D6CF7F
:10276000508190959523E3CFDF91CF911F910F91E9
:10277000FF90EF9008951F93CF93DF93EC018D8D21
:102780009E8D009721F1162F29A131E0309386020A
:10279000209385021092840210928302DC01ED9155
:1027A000FC910190F081E02D60E009958D8D9E8D6A
:1027B000DC01ED91FC910190F081E02D612F0995F4
:1027C0008D8D9E8DDF91CF911F910C941F12ADA521
:1027D000BEA59C918BA9809589238C938B8D9C8D14
:1027E000892B31F0862FDF91CF911F910C94340B00
:1027F00028E030E080E8A9A5BAA599A9462F48238A
:10280000C1F04C91942B9C93ABA5BCA59C914AA97B
:10281000942B9C93ABA5BCA54C919AA9909594231D
:102820009C9386952150310931F7DF91CF911F910B
:1028300008954C9190959423E6CFDF92EF92FF920A
:102840000F931F93CF93DF9380910D0590910E0509
:10285000892B09F4A5C020912505309126054091CA
:1028600027055091280560E074E284EF90E00E9413
:1028700051292051310941095109569547953795FC
:1028800027952093B80064E081E89CE00E9406133D
:102890008091F4049091F5048034910509F097C07B
:1028A00060E280EF94E00E94BB136091F404615EEB
:1028B00080EF94E00E94BB132091F6043091F7045E
:1028C000C901079697FD079633E0959587953A9548
:1028D000E1F72091F4043091F504829F8001839FF9
:1028E000100D929F100D1124C0910F05D09110056D
:1028F00080910D0590910E050C0F1D1F009709F496
:1029000098C02091110531E0309386022093850212
:102910001092840210928302DC01ED91FC910190EF
:10292000F081E02D60E40995EE24E394F12CDD24A0
:10293000D39480910D0590910E050C171D0709F495
:102940004FC0B0E2EB16F104D8F00E941F12809144
:102950000D0590910E0520911105D09286022093CD
:1029600085021092840210928302DC01ED91FC91A9
:102970000190F081E02D60E40995EE24E394F12CC0
:1029800080910D0590910E056991DC01ED91FC910E
:102990000190F081E02D0995BFEFEB1AFB0AC9CF3A
:1029A00080910B0590910C05892B31F080912E05BB
:1029B00090912F050E943B0BE0911F05F09120059F
:1029C0009081809124058095892380835CCF60E08D
:1029D00080EF94E00E94BB136091F404615068CFD3
:1029E0000E941F1280910D0590910E05892B09F40C
:1029F00061C02091290530912A0540912B05509105
:102A00002C0560E074E284EF90E00E94512920518F
:102A100031094109510956954795379527952093D6
:102A2000B800DF91CF911F910F91FF90EF90DF9051
:102A30000895E0911D05F0911E0580819091230578
:102A4000892B80830C171D0769F2899120910B0552
:102A500030910C05232B19F00E94340BF3CF28E0A2
:102A600030E040E8E0911905F0911A0590912105B8
:102A7000582F5423D9F05081952B9083E0911B055A
:102A8000F0911C05908150912205952B9083E09147
:102A90001B05F0911C05508190912205909595237E
:102AA0009083469521503109E9F6CCCF508190951D
:102AB0009523E3CFE0911F05F0912005808190914F
:102AC0002405892B8083ADCF1F93CF93DF93EC0137
:102AD000162F8D8D9E8D892BB1F12DA93EA94FA961
:102AE00058AD60E074E284EF90E00E9451292051DB
:102AF00031094109510956954795379527952093F6
:102B0000B80066EA111167EACE010E94BB138D8DF1
:102B10009E8D892B41F129AD3AAD4BAD5CAD60E0A6
:102B200074E284EF90E00E9451292051310941095B
:102B3000510956954795379527952093B800DF9111
:102B4000CF911F9108958B8D9C8D892B21F08EAD97
:102B50009FAD0E943B0BEFA5F8A990818CA98095B1
:102B600089238083CECFEFA5F8A980819CA9892BEA
:102B70008083E5CF90E080E00895FC018481958119
:102B8000228133812817390771F0860F971F6081E2
:102B900071810E9473290680F781E02DE80FF91FEB
:102BA000808190E008958FEF9FEF0895FC0184816C
:102BB0009581228133812817390741F0860F971FAD
:102BC000608171810E947329958384830895FC013B
:102BD000462F22813381C9010196608171810E9453
:102BE0007329648175818617970781F0A681B78163
:102BF000A20FB31F4C9382819381019660817181F2
:102C00000E9473299383828380E008958FEF089553
:102C1000EF92FF920F931F93CF93DF937C01062FC8
:102C200010E0B80186E594E00E94E715D0E0C0E02E
:102C3000C017D10758F4F701EC0FFD1F649170E045
:102C400086E594E00E94E7152196F2CFDF91CF91BF
:102C50001F910F91FF90EF900895CF93DF93FC01A8
:102C6000C281D38184819581C817D907C9F0A68113
:102C7000B781A80FB91F2C910196608171810E94C4
:102C80007329C817D90739F095838483822F90E080
:102C9000DF91CF9108951582148213821282F6CFAC
:102CA0008FEF9FEFF5CFFC01608171818481958169
:102CB0009B01281B390B82819381820F931F0E94F5
:102CC000732908958091AE018823B9F08091AD01F8
:102CD000882399F06CE08AED91E00E94081667E085
:102CE00083ED91E00E94081667E08CEC91E00E9471
:102CF000081661E08AE00C94DB0660E08AE00E943E
:102D0000DB0667E086EE91E00C9408168F929F92A6
:102D1000AF92BF92CF92DF92EF92FF924B015C0194
:102D20000E9445076B017C0124E0C21AD108E1082A
:102D3000F1080E9445076C197D098E099F096815E5
:102D400079058A059B05A8F3FF90EF90DF90CF905F
:102D5000BF90AF909F908F900895DC01ED91FC9112
:102D60000190F081E02D0994809144048F3F11F48B
:102D70002D98089560E00C94DB06882349F080913B
:102D800044048F3F11F42D9A089561E00C94DB0602
:102D90000C94B416CF93DF93EC0181E00E94BD1632
:102DA000299ABE0190E080E00E94861629980E9430
:102DB000B416DF91CF910C94B4168F929F92AF927C
:102DC000BF92CF92DF92EF92FF92CF934B015C01C3
:102DD000219A8FEF88169806A806B806C1F4219AA2
:102DE00080E093E20E94CA1660EC78E080E090E018
:102DF0000E94861680E392E0CF91FF90EF90DF90E3
:102E0000CF90BF90AF909F908F900C94CA1680E0A7
:102E100093E20E94CA1660E871E180E090E00E94AF
:102E20008616C0E2C12CD12CE12C90E8F92ED501F8
:102E3000C4018C219D21AE21BF21892B8A2B8B2B94
:102E400089F080E392E00E94CA1660E976E080E0B3
:102E500090E00E948616F694E794D794C794C150E8
:102E600031F7C8CF80E392E00E94CA1660E372E0B7
:102E700080E090E0EECFFB0101900020E9F7319770
:102E8000AF01461B570BDC01ED91FC910280F381F1
:102E9000E02D09948F929F92AF92BF920F931F9350
:102EA000CF93DF93CDB7DEB7A1970FB6F894DEBF0F
:102EB0000FBECDBF19A2423008F44AE08E010F5D6B
:102EC0001F4F842E912CB12CA12CA50194010E949E
:102ED0005129E62FB901CA01EA3004F5E05DD801B5
:102EE000EE938D01232B242B252B79F790E080E0A6
:102EF000109729F0BD0180EF94E00E943B17A19646
:102F00000FB6F894DEBF0FBECDBFDF91CF911F91FA
:102F10000F91BF90AF909F908F900895E95CDFCFA5
:102F2000CF93DF93682F70E090E080E04AE00E944A
:102F30004A17EC0160EA71E080EF94E00E943B17D1
:102F40008C0F9D1FDF91CF9108950F931F93CF9307
:102F5000DF93EC010E94AC078C0160EA71E0CE01C6
:102F60000E943B17800F911FDF91CF911F910F910E
:102F70000895CF9320EB34E0F90101900020E9F7A8
:102F80009F01215B3440C091AB0433274C2F50E0AC
:102F9000BA0161507109261B370B3093A6042093A8
:102FA000A504682F70E060557B4F88E191E00E9496
:102FB000B72A80911801803219F486E880931801AD
:102FC000CB5FC0931301EC2FF0E0319620E090E04E
:102FD000A92FB0E0AE5EBE4F4C9124279F5FC9176A
:102FE000B8F7EE5EFE4F20836091130170E06E5FD4
:102FF0007F4F8EE594E00E94E715C0E02C2F30E073
:103000008091130190E00196821793075CF02E5E89
:103010003E4FF901608170E08EE594E00E94E71573
:10302000CF5FECCFCF9108952091F6043091F70453
:10303000C901079697FD079623E0959587952A95F0
:10304000E1F72091F4043091F504829FA001839F61
:10305000500D929F500D112470E060E080910F059B
:10306000909110050C94C02A0E94B22A85ED80939D
:10307000BC008091F0019091F101A091F201B0911A
:10308000F3010796A11DB11D23E0B695A79597956D
:1030900087952A95D1F72091BC0024FD03C010929A
:1030A000390208954091F0015091F1016091F201CF
:1030B0007091F301452B462B472B69F30097A1052F
:1030C000B10541F02AE22A95F1F700C00197A10964
:1030D000B109E1CF8091EF010C9479111F93CF9347
:1030E000DF93EC01162F0E943B29181739F0612F4E
:1030F000CE01DF91CF911F910C944329DF91CF91A5
:103100001F9108950C943B298BE090E00E94821857
:10311000282F30E030930B0120930A018330A1F077
:1031200028F4813041F0823059F00895843081F0E4
:10313000853091F008956AE18AE491E00C940816D4
:103140006AE182EB91E0FACF6AE188E991E0F6CF9B
:103150006AE18EE791E0F2CF6AE184E691E0EECF9A
:10316000CF93DF9390E080E00E948218C82FD0E0D8
:10317000D0930901C09308018AE090E00E94821870
:10318000282F30E03093070120930601219739F46E
:10319000833019F180F48130B1F08230D1F08AE0CF
:1031A00090E00E94821890E09093070180930601BE
:1031B000DF91CF9108958430A1F0853081F76AE1E5
:1031C00084E691E003C06AE18AE491E00E94081677
:1031D000E6CF6AE182EB91E0F9CF6AE188E991E01C
:1031E000F5CF6AE18EE791E0F1CF90E080E00E94B8
:1031F0008218282F30E0309305012093040183309A
:10320000D9F028F4813049F0823069F00895853092
:1032100019F1D0F08730E9F008951092AD010E94C5
:1032200062160C9484181092AD010E9462166AE135
:1032300080E391E00C9408161092AD010E94621692
:103240006AE186E191E0F6CF6AE18CEF90E00E94BE
:1032500008161092AD0108C06AE182EE90E00E946B
:10326000081681E08093AD010C9462164F925F9234
:103270006F927F92AF92BF92CF92DF92EF92FF92C6
:103280000F931F93CF93DF93CDB7DEB768970FB639
:10329000F894DEBF0FBECDBF7C01FC01D080A280C0
:1032A000C3800481B58016810E949C074090A401D0
:1032B0005090A5016090A6017090A7019B01AC0100
:1032C000241935094609570929013A0130E1431605
:1032D00037E253066104710468F06093A4017093AF
:1032E000A5018093A6019093A70165E088E690E090
:1032F0000E94081645E050E06DED70E0C7010E94A5
:103300002E29892B29F466E087ED90E00E940816AB
:1033100046E050E061ED70E0C7010E942E29892B44
:1033200019F481E08093AE018091790281110AC085
:1033300066E083E59CE00E9408160E94F51881E093
:103340008093790245E050E06CEC70E0C7010E9488
:103350002E29892B29F466E086EC90E00E9408165D
:1033600045E050E060EC70E0C7010E942E29892BF7
:1033700011F40E94F51840E8D41230C35FEBA51297
:1033800030C388E1C8122DC3B0926B02802F90E049
:10339000880F991F90936D0280936C0245E0489FBF
:1033A0009001499F300D11242C5F3F4F43E036952B
:1033B00027954A95E1F730937302209372024FE00C
:1033C000429FC001439F900D1124839666E470E0F4
:1033D0000E947329615F7F4F8091AB019091AC0196
:1033E000680F791F6432710514F063E270E077FDB5
:1033F00060E06093110111E01093780261E081E1D7
:103400000E94DB068091AA01811104C00E94F51878
:103410001093AA0168960FB6F894DEBF0FBECDBF19
:10342000DF91CF911F910F91FF90EF90DF90CF90A0
:10343000BF90AF907F906F905F904F900895153040
:1034400009F4F2C0163031F766E08AE990E00E9494
:1034500008168091AD01882309F441C18091AE0125
:10346000882309F43CC167E083E990E017C11A3072
:1034700009F4B1C108F046C0183009F435C119305B
:1034800049F690E080E00E94821890E09093090154
:1034900080930801019709F060C16FE470EB8EE43E
:1034A00091E60E94DD1685E090E090930301809301
:1034B000020180910A0190910B01019686309105DD
:1034C0000CF048C190930B0180930A0160910A01AE
:1034D0008BE090E00E946E1868960FB6F894DEBFFD
:1034E0000FBECDBFDF91CF911F910F91FF90EF9055
:1034F000DF90CF90BF90AF907F906F905F904F9094
:103500000C9484181B3009F4B6C11C3009F082CF2A
:1035100066E087E890E00E94081665E97AE68EE4A6
:1035200091E67CC21A3209F4DBC110F5173209F4B6
:103530002FC298F4133209F4CEC1163209F06ACFC3
:103540008091AD01882321F08091AE018111A8C046
:103550006FE870E78EE491E661C2183209F425C283
:103560006FE470EB8EE491E6193209F457C252CF42
:103570001D3209F4ECC158F41B3209F4E3C165ECC7
:103580007AE38EE491E61C3209F448C243CF1A3440
:1035900009F429C11E3409F03DCF60E08AE0689645
:1035A0000FB6F894DEBF0FBECDBFDF91CF911F9154
:1035B0000F91FF90EF90DF90CF90BF90AF907F90F2
:1035C0006F905F904F900C94DB0666E08AEB90E082
:1035D0000E94081667ED78E28EE491E60E94DD16FF
:1035E000809171028823E1F0809170028823C1F0FC
:1035F00080911001833218F48F5F809310018091C5
:103600001101833268F42091AB013091AC012F5F3E
:103610003F4F3093AC012093AB018F5F809311013A
:1036200081E080937802F6CE66E084EB90E00E9421
:10363000081667E578EA8EE491E60E94DD1680912F
:103640007102882369F380917002882349F3809185
:103650001001882319F0815080931001809111018D
:103660008823F1F22091AB013091AC012150310956
:103670003093AC012093AB018150D0CF66E08EEA4D
:1036800090E00E9408168091AD0167E08823F1F078
:103690008091AE018823D1F087EA90E00E9408165D
:1036A00068960FB6F894DEBF0FBECDBFDF91CF9105
:1036B0001F910F91FF90EF90DF90CF90BF90AF9050
:1036C0007F906F905F904F900C94621680EA90E02C
:1036D0000E94081667EB78E48EE491E69FC167E3E9
:1036E00078EC8EE491E69AC166E08DE890E00E9465
:1036F00008166FEA70E58EE491E60E94DD1680916F
:1037000004019091050101968630910504F590938E
:103710000501809304016091040190E080E00E9423
:103720006E1868960FB6F894DEBF0FBECDBFDF915E
:10373000CF911F910F91FF90EF90DF90CF90BF90AE
:10374000AF907F906F905F904F900C94F51881E050
:1037500090E0DDCF81E090E0B5CE90E080E00E9487
:10376000821890E09093090180930801029709F074
:1037700051CE809106019091070101969093070127
:103780008093060120910201309103012817390727
:1037900034F481E090E090930701809306016091FA
:1037A00006018AE090E00E946E1868960FB6F894C1
:1037B000DEBF0FBECDBFDF91CF911F910F91FF9064
:1037C000EF90DF90CF90BF90AF907F906F905F9021
:1037D0004F900C94B0188091A90181111BCE81E00B
:1037E0008093A80117CE8091A901882329F0109217
:1037F000A9011092A8010ECE8091A8018823C9F3D7
:10380000809100019091010101968630910574F537
:1038100090930101809300016091000188E290E0A3
:103820000E946E1888E290E00E94821890E09093C7
:1038300001018093000128E1E8E3F1E0DE01119647
:1038400001900D922A95E1F7880F991F880F991F13
:10385000E1E0F0E0EC0FFD1F8E0F9F1FFC01608187
:103860007181828193810E94DD16C3CF1092010184
:1038700010920001D1CF65E77AE88EE491E6CEC0E0
:1038800061E08AE00E94DB068CE00E94B206892B90
:1038900029F060E08CE00E94DB0643CF61E08CE021
:1038A0000E94DB066AE18DE690E068960FB6F89418
:1038B000DEBF0FBECDBFDF91CF911F910F91FF9063
:1038C000EF90DF90CF90BF90AF907F906F905F9020
:1038D0004F900C9408166FE170EE8EE491E69EC056
:1038E0008091A901811196CD91E09093A901109248
:1038F000A801809171028927809371028823B9F011
:103900001092AC011092AB011092700283E280938E
:103910006F028FE080936E020E949C0760936702A3
:10392000709368028093690290936A0279CE109234
:10393000AC011092AB011092700210926F021092C3
:103940006E026ECE6FE570EA8EE491E667C061E0CC
:1039500090E080E00E946E1861E08AE090E00E94B2
:103960006E1861E08BE090E00E946E1860E08EE1DE
:1039700090E00E946E1860E088E290E00E946E186D
:1039800060E08CE890E00E946E180E94F5180DCF60
:103990008091AD01882321F08091AE01811180CE0C
:1039A0006FE070EF8EE491E639C062E090E080E075
:1039B00068960FB6F894DEBF0FBECDBFDF91CF91F2
:1039C0001F910F91FF90EF90DF90CF90BF90AF903D
:1039D0007F906F905F904F900C946E1820ECD212F5
:1039E00019CDF1E3CF1216CD61E085E00E94DB0630
:1039F0001E3009F445CF08F095CD173009F43ECEBE
:103A000008F035CD143009F4E0CD08F018CD67E9A1
:103A100078E68EE491E6133009F0FCCC68960FB698
:103A2000F894DEBF0FBECDBFDF91CF911F910F91F4
:103A3000FF90EF90DF90CF90BF90AF907F906F900E
:103A40005F904F900C94DD161F920F920FB60F925D
:103A500011242F933F938F939F93AF93BF938091A4
:103A60007B0290917C02A0917D02B0917E02309108
:103A70007A0223E0230F2D3758F50196A11DB11DC1
:103A800020937A0280937B0290937C02A0937D0224
:103A9000B0937E0280917F0290918002A09181027A
:103AA000B09182020196A11DB11D80937F02909377
:103AB0008002A0938102B0938202BF91AF919F9147
:103AC0008F913F912F910F900FBE0F901F901895DF
:103AD00026E8230F0296A11DB11DD2CF1F920F928F
:103AE0000FB60F9211242F933F934F935F936F93D1
:103AF0007F938F939F93AF93BF93EF93FF93E09147
:103B00000E01F0910F010995FF91EF91BF91AF91D7
:103B10009F918F917F916F915F914F913F912F91E5
:103B20000F900FBE0F901F9018951F920F920FB617
:103B30000F9211242F933F934F935F936F937F9333
:103B40008F939F93AF93BF93EF93FF93E0910C01FB
:103B5000F0910D010995FF91EF91BF91AF919F9168
:103B60008F917F916F915F914F913F912F910F9026
:103B70000FBE0F901F9018951F920F920FB60F92C5
:103B800011242F933F934F935F936F937F938F9362
:103B90009F93AF93BF93EF93FF9387E892E00E94C8
:103BA0004E08FF91EF91BF91AF919F918F917F91BF
:103BB0006F915F914F913F912F910F900FBE0F909A
:103BC0001F9018951F920F920FB60F9211242F93EA
:103BD0008F939F93EF93FF93E0919702F091980258
:103BE0008081E0919D02F0919E0282FD1BC0908138
:103BF0008091A0028F5F8F732091A102821741F004
:103C0000E091A002F0E0E957FD4F958F8093A0026C
:103C1000FF91EF919F918F912F910F900FBE0F9079
:103C20001F9018958081F4CF1F920F920FB60F92BC
:103C300011242F933F934F935F936F937F938F93B1
:103C40009F93AF93BF93EF93FF938091B900887FC9
:103C5000803609F44AC0F0F5883209F4A7C018F597
:103C6000803109F49BC0B8F4882309F4F9C0883086
:103C700009F494C0FF91EF91BF91AF919F918F9103
:103C80007F916F915F914F913F912F910F900FBE58
:103C90000F901F901895883109F488C0803251F731
:103CA0008093380214C0803409F49DC040F48033FE
:103CB000B9F38833F9F68093380285ECB0C08035CB
:103CC00009F485C0883509F496C0883499F60E94B5
:103CD0003618D0CF883909F48CC038F5883729F0E8
:103CE00050F4883611F0803729F683E0809339024A
:103CF0001092370257C0883809F47BC0803919F018
:103D0000803809F0B7CF80913702803208F071C057
:103D1000E091370281E08E0F809337028091BB00E3
:103D2000F0E0E95EFD4F80833DC0803B39F0E0F478
:103D3000803A09F479C0883A09F09CCF84E08093F6
:103D400039021092160210921502E0916202F0916F
:103D5000630209958091150281110FC081E0809363
:103D600015021092F50109C0803C09F4A6CF883CE9
:103D700009F4A3CF883B09F07DCFE091160281E0E2
:103D80008E0F80931602F0E0EB50FE4F80818093FF
:103D9000BB00909116028091150229C080915E02AD
:103DA0008093BB0085EC8093BC0064CF90915D0252
:103DB00080915C02981758F5E0915D0281E08E0FCA
:103DC00080935D02F0E0E45CFD4F8081E9CFE091FB
:103DD0005D0281E08E0F80935D028091BB00F0E078
:103DE000E45CFD4F808390915D0280915C029817A6
:103DF000C8F285E8D8CFE0915D0281E08E0F809314
:103E00005D028091BB00F0E0E45CFD4F8083809117
:103E10003B0281115CCF81E080933A0284EA809377
:103E2000BC001092390226CF85EC8093BC00109222
:103E3000390280913702803230F4E0913702F0E0AD
:103E4000E95EFD4F10826091370270E0E091600200
:103E5000F091610287E192E00995109237020ACF52
:103E60001092380234CF1F920F920FB60F92112486
:103E70002F933F934F935F936F937F938F939F9372
:103E8000AF93BF93CF93EF93FF93E0913203F09101
:103E90003303C08180913403C8238091350390910E
:103EA000360320913503309136032F3F3F4F29F0E1
:103EB00001969093360380933503209130032111AE
:103EC00015C0C1114BC0813A910558F010923F03C3
:103ED000909342038093410381E080934003809359
:103EE0003003109236031092350338C0213099F414
:103EF000CC23A1F1E09140032E0F20934003F0E08A
:103F0000E05DFC4F8F3F910519F010F08FEF90E0CE
:103F1000838B82E0E4CF223009F047C0E091400378
:103F2000813A910510F4E73CA0F1E83C18F081E0FB
:103F300080933F0380914103909142039093380412
:103F400080933704E093360483E080933003E0915C
:103F50003703F0913803309709F0099580914504B3
:103F6000882329F081E0C11180E00E94BD16FF91F5
:103F7000EF91CF91BF91AF919F918F917F916F9171
:103F80005F914F913F912F910F900FBE0F901F9017
:103F90001895C111E3CF91E09E0F90934003F0E09C
:103FA000E05DFC4F838B81E09ACF2330B9F6C111DD
:103FB000D5CF97CF1F920F920FB60F9211242F9348
:103FC0003F934F935F936F937F938F939F93AF93A1
:103FD000BF93EF93FF9381E08093660260E08DE0F2
:103FE0000E94DB06E1EBF0E08081887F8083FF9117
:103FF000EF91BF91AF919F918F917F916F915F9161
:104000004F913F912F910F900FBE0F901F901895D9
:104010001F920F920FB60F9211242F933F934F933D
:104020005F936F937F938F939F93AF93BF93EF9320
:10403000FF9380E00E94B2060197D9F481E00E94CC
:10404000B2060197B1F48091B10087608093B1000E
:10405000FF91EF91BF91AF919F918F917F916F9160
:104060005F914F913F912F910F900FBE0F901F9036
:10407000189580E00E94B206892B51F781E00E94DA
:10408000B206019729F71092660261E08DE00E9466
:10409000DB068091B100887FD9CFFC0186819781B2
:1040A000009711F00C94292A08958EE594E00E945F
:1040B0004D2086E594E00E944D208EE494E00E941D
:1040C0004D2088E791E09093F1048093F004809173
:1040D0000F0590911005009711F00C94292A08956E
:1040E0000F931F93CF93DF93EC018B017983688348
:1040F0001D821C821B821A82CB010E948D299F8304
:104100008E83A80170E060E0DF91CF911F910F9145
:104110000C94C02AEF92FF920F931F93CF93DF93DB
:10412000E7E8F2E01382128288EE93E0A0E0B0E0CC
:1041300084839583A683B78324E531E0318320838C
:1041400025EC30E03587248724EC30E0378726875C
:1041500020EC30E0318B208B21EC30E0338B228B54
:1041600022EC30E0358B248B26EC30E0378B268B2D
:10417000118E128E138E148E24E2E22E23E0F22E84
:10418000F7011382128284839583A683B78386E620
:1041900091E0918380831FEF10934404E0E3F3E008
:1041A000118201E0048389E290E093838283509836
:1041B000C6E6D4E01CAA0E949C0760934A04709350
:1041C0004B0480934C0490934D040E949C07609391
:1041D00046047093470480934804909349041986D9
:1041E0001A861B8618861F821E821D8262E080E06E
:1041F0000E94090761E084E00E94090761E084E011
:104200000E94DB06E0EBF0E010821092B1008DE935
:104210008093B300808182608083E0E7F0E080815A
:1042200082608083E8E6F0E0808184608083EDE650
:10423000F0E080818160808319821A8280ED97E0AE
:104240009AAF89AF88EE93E09CAF8BAF88EC90E09B
:104250009EAF8DAF82E08093AC041092A6041092C2
:10426000A5048BE08093AB041092AD041092AE04D1
:104270001092AF040E949C076093A7047093A80457
:104280008093A9049093AA04E0EFF4E013821282D1
:1042900020E830E03583248380E290E097838683B2
:1042A0003187208793878287168A1586148617861A
:1042B0001686058B048B8FEF9FEF938B828B918BF0
:1042C000808B078B108E128E118E88E791E0918380
:1042D0008083148E138EF68EE58E10A2178E14A393
:1042E00015A316A317A310A780E89AE1A6E0B0E0F3
:1042F00085AB96ABA7ABB0AF80EA96E8A1E0B0E0A3
:1043000081AF92AFA3AFB4AF80E586AF17AE0E9486
:104310009C0760934A0470934B0480934C049093E1
:104320004D040E949C076093460470934704809359
:1043300048049093490460E870E08EE494E00E94A1
:10434000702060E470E086E594E00E94702060E4F4
:1043500070E08EE594E0DF91CF911F910F91FF9077
:10436000EF900C947020789484B5826084BD84B5FD
:10437000816084BD85B5826085BD85B5816085BD60
:1043800080916E00816080936E0010928100809118
:1043900081008260809381008091810081608093A0
:1043A0008100809180008160809380008091B100C5
:1043B00084608093B1008091B00081608093B000F0
:1043C00080917A00846080937A0080917A00826084
:1043D00080937A0080917A00816080937A00809146
:1043E0007A00806880937A001092C1001092650272
:1043F0001092640210928402109283020E945B1158
:1044000089EA97E090936302809362028AEA97E0D8
:10441000909361028093600268EC70E080E090E02D
:104420000E946A0780910F0590911005892B41F534
:104430002091F6043091F704C901079697FD07967D
:10444000B3E095958795BA95E1F72091F404309102
:10445000F504AC01429FC001439F900D529F900D07
:1044600011240E948D299093100580930F05892BAC
:1044700039F461EE7BE087E892E00E94A517FFCF58
:104480000E9414182091F6043091F7048091F404EE
:104490009091F504B901213231050CF423C2605426
:1044A000710977FF02C06F5F7F4F759567958255E1
:1044B000910997FD019600E410E022E530E04FEE0F
:1044C00058E0959587950E94251082E0809312050B
:1044D00080910D0590910E05892B09F416C28CE38D
:1044E000809311051092650210926402109284026A
:1044F000109283020E945B1189EA97E09093630215
:10450000809362028AEA97E090936102809360024E
:104510008091180587FD1EC061E00E94090761E0D7
:10452000809118050E94DB0661E070E080E090E079
:104530000E946A0760E0809118050E94DB066AE02D
:1045400070E080E090E00E946A0761E080911805C9
:104550000E94DB0680910D0590910E05892B09F4D0
:1045600093C2209125053091260540912705509151
:10457000280560E074E284EF90E00E945129205108
:10458000310941095109569547953795279520934B
:10459000B80064E08BE097E00E9406136091F60497
:1045A000615080EF94E00E94BB1364E087E097E0E5
:1045B0000E9406138091120560E1813009F064E1E8
:1045C00080EF94E00E94BB1364E083E097E00E94D8
:1045D00006138FE880932D058091F4049091F504E3
:1045E0008038910509F067C28091F6049091F70434
:1045F0008034910509F06FC280911205813009F075
:104600007DC28FE980932D05C2E16AED80EF94E0D1
:104610000E94BB136C2F80EF94E00E94BB1361E8F3
:1046200080EF94E00E94BB1360912D0580EF94E031
:104630000E94BB1369ED80EF94E00E94BB13809150
:10464000120562E2813009F061EF80EF94E00E9490
:10465000BB1366E08DEF96E00E94061380910D0576
:1046600090910E05892B09F44BC2209129053091B8
:104670002A0540912B0550912C0560E074E284EFEF
:1046800090E00E9451292051310941095109569564
:104690004795379527952093B8000E941418C1E0DC
:1046A000C0930405C093050581E090E09093030555
:1046B0008093020590930105809300051092FD04FC
:1046C0001092FC041092FF041092FE04C09308059F
:1046D00063ED7BE080EF94E00E94A51761EC7BE046
:1046E00080EF94E00E94A5176FEA7BE080EF94E0F2
:1046F0000E94A5170E941D1461E085E00E94090731
:1047000061E086E00E94090760E08AE00E940907F4
:1047100061E08BE00E94090761E08CE00E940907DC
:1047200062E084E10E94090761E08DE00E940907D0
:10473000E0919702F0919802D2E0D083E091930249
:10474000F09194021082E0919502F091960280E13E
:10475000808310929F02E0919B02F0919C0286E080
:104760008083E0919902F0919A0280818061808338
:10477000E0919902F0919A02808188608083E091B3
:104780009902F0919A02808180688083E091990279
:10479000F0919A0280818F7D808361E085E00E94A4
:1047A000DB06C09386028FE280938502109284021A
:1047B000109283026FE784E293E00E94F01184E29A
:1047C00093E00E941F1287E892E090936A0480931E
:1047D0006904E0919702F0919802D083E0919302EE
:1047E000F09194021082E0919502F09196028FEC84
:1047F000808310929F02E0919B02F0919C0286E2DE
:104800008083E0919902F0919A0280818061808397
:10481000E0919902F0919A02808188608083E09112
:104820009902F0919A02808180688083E0919902D8
:10483000F0919A0280818F7D80838CED95E090933A
:10484000A00480939F0488EE93E09093A204809349
:10485000A10488EC90E09093A4048093A304D093E7
:10486000AC0486E399E190939E0480939D0461E0FB
:104870008DE00E94090722E0422E512C01E010E059
:1048800034E0632E712C43E0A42EB12CC1E090E003
:10489000292E90E0392E8091790281110FC068EEA7
:1048A00073E080E090E00E946A0766E083E59CE0A8
:1048B0000E9408160E94F518C0937902E0916B04DB
:1048C000F0916C04E830F10508F026C1E659FB4D83
:1048D0000C9487298A25602676269726C026D52619
:1048E000E9260A276052710977FF02C06F5F7F4F88
:1048F000759567958357910997FD019600E210E041
:1049000023E730E04FE057E0DCCD61E08091160511
:104910000E94090761E0809117050E9409078091B4
:104920001605082E000C990BFC01E157F34FE4919A
:10493000F0E0EE0FFF1FED59F34F259134913093C6
:104940001E0520931D05FC01ED55F34FE491E09306
:10495000230580911705082E000C990BFC01E157E7
:10496000F34FE491F0E0EE0FFF1FED59F34FA591E7
:10497000B491B0932005A0931F05FC01ED55F34FB2
:10498000E491E09324058C91E82BEC9380910B0546
:1049900090910C05892B09F434C0CFB7F89480911D
:1049A0005F02811127C0E9E9FCE08491EDEAFCE0B7
:1049B0009491E82FF0E0EE0FFF1FE75AF34FA59117
:1049C000B491EC91E92321F461E08AE00E94DB06D6
:1049D00061E08AE00E9409078CB580618CBD8CB5CE
:1049E00080648CBD61E08DE00E94090761E08BE08E
:1049F0000E94090780915F028F5F80935F02CFBFA3
:104A000087CD61E0809114050E94090761E08091E3
:104A100015050E94090780911405082E000C990BBA
:104A2000FC01E157F34FE491F0E0EE0FFF1FED5969
:104A3000F34F2591349130931A0520931905FC0109
:104A4000ED55F34FE491E093210580911505082E73
:104A5000000C990BFC01E157F34FE491F0E0EE0FED
:104A6000FF1FED59F34FA591B491B0931C05A0938E
:104A70001B05FC01ED55F34FE491E09322058C9169
:104A8000E095E823EC9344CD80910B0590910C05C3
:104A9000892B31F080912E0590912F050E943B0BC0
:104AA000E0911F05F091200590818091240580956B
:104AB000892380836ECD8036910589F48091F60438
:104AC0009091F704409739F480911205813029F4D0
:104AD00080E180932D05C2E098CD8FEAFACF803433
:104AE0009105C9F78091F6049091F704809799F7A2
:104AF00080911205813011F480E184CD8FEC82CD5C
:104B0000E0911F05F0912005808190912405892B6B
:104B10008083C3CD1092AD04809166028823E9F0B2
:104B20008EE594E00E94531618161906B4F48EE52B
:104B300094E00E942D166C0180E00E94B20601975D
:104B400039F4F12CE12CF3E1CF16D10408F488C13B
:104B5000B6018EE594E00E94D6158091690490918B
:104B60006A04DC01ED91FC910084F185E02D09954A
:104B7000892B81F08091690490916A04DC01ED91A8
:104B8000FC910284F385E02D0995BC018EE494E04C
:104B90000E94E71580916D0490916E04823091051A
:104BA00009F4B3C108F070C1009709F47BC1019703
:104BB00009F48DC1809166028823D1F186E594E0E5
:104BC0000E945316181619069CF50E949C07C09067
:104BD0004604D0904704E0904804F09049046C19D2
:104BE0007D098E099F096A3071058105910500F1E3
:104BF00086E594E00E942D166C0180E00E94B206CA
:104C0000019739F4F12CE12CB1E2CB16D1040CF46C
:104C1000FEC1B60186E594E00E94D6150E949C076D
:104C2000609346047093470480934804909349042A
:104C300080916704882371F00E949C0760E084E003
:104C40000E94DB0670E060E08091690490916A0444
:104C50000E94AD1680917102882309F401C2C090B0
:104C60006702D0906802E0906902F0906A02809139
:104C700070028111A7C20E949C076C197D098E09E0
:104C80009F09663971058105910508F4E9C1D09144
:104C90006F02DD2309F4CFC167E578EA8EE491E67F
:104CA0000E94DD16D150D0936F020E949C07609342
:104CB0006702709368028093690290936A02CEC182
:104CC0001092AF041092AE0480E00E94B917509287
:104CD0006C0440926B040E949C076093A70470933D
:104CE000A8048093A9049093AA0416CF0E949C075D
:104CF000C090A704D090A804E090A904F090AA0462
:104D0000AB01BC014C195D096E097F0980919F04BC
:104D10009091A004B0E0A0E0481759076A077B070C
:104D200008F4FACEB0926C04A0926B04F5CE2091F8
:104D3000AE048091A5049091A6042817190680F46A
:104D40002F5F2093AE048091AF0491E0980F909371
:104D5000AF040E94B91770926C0460926B04BBCFD1
:104D600085E090E090936C0480936B041092AF0404
:104D70001092AE048091AD048F5F8093AD04CCCED1
:104D80000E949C07C090A704D090A804E090A904BA
:104D9000F090AA04AB01BC014C195D096E097F09B2
:104DA0008091A3049091A404B5CF9091AD0480911B
:104DB000AC04981738F4A6E0B0E0B0936C04A0936C
:104DC0006B0489CFE7E0F0E0F0936C04E0936B04B0
:104DD00082CF0E949C07C090A704D090A804E090C6
:104DE000A904F090AA04AB01BC014C195D096E093D
:104DF0007F098091A1049091A204B0E0A0E048173F
:104E000059076A077B0708F487CE10936C04009358
:104E10006B0482CE0E949C07C090A704D090A80487
:104E2000E090A904F090AA04AB01BC014C195D0903
:104E30006E097F098091A1049091A204B0E0A0E0E6
:104E4000481759076A077B0708F466CE1092AF042B
:104E500080E00E94B91710926C0410926B045CCE33
:104E60008090690490906A04CE14DF0409F475CE32
:104E70008EE594E00E942D16BC01C4010E94AD167F
:104E80002FEFE21AF20AECCF8330910509F477C0D4
:104E900061E070E0049709F08DCE8EE494E00E940A
:104EA000D615B0C08EE494E00E9453161816190669
:104EB0000CF080CE70E060E08EE494E00E94BD15BE
:104EC00080936F0410936E0400936D0473CE8EE490
:104ED00094E00E94531602970CF46CCE61E070E0EF
:104EE0008EE494E00E94BD1580937004835082325A
:104EF00028F450926E0440926D045CCE61E070E044
:104F00008EE494E00E94D61555CEC0907004D12C4A
:104F10004601BFEF8B1A9B0A8EE494E00E94531661
:104F2000881699060CF046CED0E0F12CE12CB701A2
:104F30008EE494E00E94BD15D827EFEFEE1AFE0A2A
:104F4000CE14DF04A4F7B4018EE494E00E94BD15F2
:104F5000D817190679F40E949C0760934A0470934D
:104F60004B0480934C0490934D04B0926E04A09235
:104F70006D0420CE70926E0460926D041BCE809101
:104F80006F04982F9F77903521F0982F9F7B903852
:104F9000C9F486E6E82E84E0F82E970126563440C0
:104FA000FFEFEF1AFF0A8091700490E001968217DC
:104FB0009307FCF08EE494E00E942D16D7011B9617
:104FC0008C93EBCF893729F3982F9D7F983609F37F
:104FD0008F33F9F28831E9F2982F9F7D983CC9F21E
:104FE0006091700470E06E5F7F4F803B09F055CF99
:104FF000D0CFC0939A04E0919D04F0919E0482E783
:1050000094E0099510926E0410926D04D3CDEC14C7
:10501000FD040CF003CE8090690490906A0486E54C
:1050200094E00E942D16BC01C4010E94AD16EFEF62
:10503000EE1AFE0AECCFD0916E02DD2351F067ED3F
:1050400078E28EE491E60E94DD16D150D0936E0294
:105050002CCEFFE0F0931001C0937002C093780251
:1050600080917802882309F491C00E949C07C09027
:105070007402D0907502E0907602F09077026C197D
:105080007D098E099F09643671058105910508F433
:105090007DC00E949C076093740270937502809398
:1050A000760290937702109278020E941418C093AF
:1050B0000405C093050510930305009302051093A2
:1050C0000105009300051092FD041092FC0410925B
:1050D000FF041092FE046BE47CE080EF94E00E94F9
:1050E000AC07609172027091730290E080E04AE038
:1050F0000E944A1766E47CE080EF94E00E94A517C6
:105100006DE37CE080EF94E00E94AC0760911101B8
:1051100070E090E080E04AE00E944A1780917102BE
:10512000811177C061E37CE080EF94E00E94A517D5
:1051300067E07CE080EF94E00E94AC0760916C0235
:1051400070916D0290E080E04AE00E944A1761E0B1
:105150007CE080EF94E00E94A5176BEF7BE080EF8E
:1051600094E00E94AC0760916B0224E6629FB0015C
:10517000112490E080E04AE00E944A1760EA71E062
:1051800080EF94E00E943B170E941D140E949C0730
:1051900061347F418105910548F08BE00E94B206A1
:1051A000019721F460E08BE00E94DB0621143104BA
:1051B00009F471CB0E943A08882309F467CB0E9456
:1051C000000064CB0E949C076C197D098E099F0921
:1051D000623371058105910508F442CFD091100129
:1051E00080911101D81750F467ED78E28EE491E6D2
:1051F0000E94DD16DF5FD093100157CD8D1708F0A8
:105200002FCF67E578EA8EE491E60E94DD16D15053
:10521000F2CF80917002811118C080916F028823B3
:1052200059F066E27CE080EF94E00E94AC07809148
:105230006F020E9490177CCF6BE17CE080EF94E0DE
:105240000E94AC0780916E02F4CF60E17CE080EFB9
:1052500094E00E94AC0780911001EBCFFB01DC01D0
:1052600004C08D910590801921F441505040C8F739
:10527000881B990B0895F999FECF92BD81BDF89ACC
:10528000992780B50895262FF999FECF1FBA92BDB0
:1052900081BD20BD0FB6F894FA9AF99A0FBE019617
:1052A0000895A1E21A2EAA1BBB1BFD010DC0AA1F67
:1052B000BB1FEE1FFF1FA217B307E407F50720F07F
:1052C000A21BB30BE40BF50B661F771F881F991FFA
:1052D0001A9469F760957095809590959B01AC0143
:1052E000BD01CF010895AA1BBB1B51E107C0AA1F36
:1052F000BB1FA617B70710F0A61BB70B881F991F77
:105300005A95A9F780959095BC01CD010895EE0FAF
:10531000FF1F0590F491E02D09940F931F93CF93F5
:10532000DF938230910510F482E090E0E091320545
:10533000F091330530E020E0B0E0A0E0309799F440
:105340002115310509F44AC0281B390B24303105D9
:10535000D8F58A819B816115710589F1FB019383E1
:105360008283FE0111C0408151810281138148175F
:105370005907E0F04817590799F4109761F0129611
:105380000C93129713961C933296CF01DF91CF9115
:105390001F910F9108950093320510933305F4CFB8
:1053A0002115310551F04217530738F0A901DB01EF
:1053B0009A01BD01DF01F801C1CFEF01F9CF909350
:1053C000330580933205CDCFFE01E20FF31F8193A9
:1053D00091932250310939832883D7CF209130050A
:1053E00030913105232B41F4209134013091350166
:1053F00030933105209330052091320130913301F3
:105400002115310541F42DB73EB740913601509139
:105410003701241B350BE0913005F0913105E2177F
:10542000F307A0F42E1B3F0B2817390778F0AC01C7
:105430004E5F5F4F2417350748F04E0F5F1F5093A4
:10544000310540933005819391939FCFF0E0E0E0E8
:105450009CCFCF93DF930097E9F0FC013297138242
:105460001282A0913205B0913305ED0130E020E0C9
:105470001097A1F420813181820F931F2091300574
:10548000309131052817390709F061C0F0933105D3
:10549000E0933005DF91CF910895EA01CE17DF0741
:1054A000E8F54A815B819E0141155105B1F7E9019B
:1054B000FB83EA8349915991C40FD51FEC17FD076F
:1054C00061F4808191810296840F951FE90199838F
:1054D0008883828193819B838A83F0E0E0E0129647
:1054E0008D919C9113970097B9F52D913C9111974F
:1054F000CD010296820F931F209130053091310526
:105500002817390739F6309751F510923305109264
:105510003205B0933105A0933005BCCFD383C2834D
:1055200040815181840F951FC817D90761F44E5FE0
:105530005F4F88819981480F591F518340838A8129
:105540009B81938382832115310509F0B0CFF093BD
:105550003305E09332059ECFFD01DC01C0CF1382FD
:105560001282D7CF81E090E0F8940C94C72AFB0117
:10557000DC0102C001900D9241505040D8F70895CF
:10558000DC0101C06D9341505040E0F7089516E0F2
:10559000CDE5D6E004C0FE010E9487292196CE35D4
:0855A000D107C9F7F894FFCF11
:1055A800010001000100010001000100AB07AB0789
:1055B8000F0FC800802342320000000000000000E6
:1055C80000000000000000000000000000000000D3
:1055D80000000000340580007D824E61BD424E61AE
:1055E8003DC24E61DD224E615DA24E619D624E61FB
:1055F800000000007008D007FD07BD082E080C0841
:10560800200800000000F011C311BA158806BC116B
:10561800A9119A1100000000790DD007BA153311AD
:10562800840A88061E10F60F1210061086108806C7
:105638003F0B6415F4093D0A3F0F220FAA0E4B0ECB
:045648000D0A000047
:00000001FF
